

Microchip Technology PIC18 LITE Macro Assembler V1.35 build -356382666 
                                                                                               Thu Apr 27 03:08:27 2017

Microchip Technology Omniscient Code Generator v1.35 (Free mode) build 201507080246
     1                           	processor	18F4550
     2                           	fnconf	rparam,??,?,0
     3                           	opt	pw 120
     4                           	opt	lm
     5                           	psect	idataCOMRAM,global,class=CODE,delta=1
     6                           	psect	cinit,global,reloc=2,class=CODE,delta=1
     7                           	psect	dataCOMRAM,global,class=COMRAM,space=1,delta=1
     8                           	psect	cstackCOMRAM,global,class=COMRAM,space=1,delta=1
     9                           	psect	text0,global,reloc=2,class=CODE,delta=1
    10                           	psect	text1,global,reloc=2,class=CODE,delta=1
    11                           	psect	text2,global,reloc=2,class=CODE,delta=1
    12                           	psect	text3,global,reloc=2,class=CODE,delta=1
    13                           	psect	text4,global,reloc=2,class=CODE,delta=1
    14                           	psect	text5,global,reloc=2,class=CODE,delta=1
    15                           	psect	text6,global,reloc=2,class=CODE,delta=1
    16                           	psect	text7,global,reloc=2,class=CODE,delta=1
    17                           	psect	text8,global,reloc=2,class=CODE,delta=1
    18                           	psect	text9,global,reloc=2,class=CODE,delta=1
    19                           	psect	text10,global,reloc=2,class=CODE,delta=1
    20                           	psect	text11,global,reloc=2,class=CODE,delta=1
    21                           	psect	text12,global,reloc=2,class=CODE,delta=1
    22                           	psect	text13,global,reloc=2,class=CODE,delta=1
    23                           	psect	text14,global,reloc=2,class=CODE,delta=1
    24                           	psect	intsave_regs,global,class=BIGRAM,space=1,delta=1
    25                           	psect	rparam,global,class=COMRAM,space=1,delta=1
    26  0000                     
    27                           	psect	idataCOMRAM
    28  007CBD                     __pidataCOMRAM:
    29                           	opt stack 0
    30                           
    31                           ;initializer for _ADDRESS_DATA_PIPE0
    32  007CBD  05                 	db	5
    33  007CBE  04                 	db	4
    34  007CBF  03                 	db	3
    35  007CC0  02                 	db	2
    36  007CC1  01                 	db	1
    37  0000                     _ADCON0	set	4034
    38  0000                     _ADCON1	set	4033
    39  0000                     _ADCON1bits	set	4033
    40  0000                     _LATB	set	3978
    41  0000                     _LATDbits	set	3980
    42  0000                     _PIR1bits	set	3998
    43  0000                     _SSPBUF	set	4041
    44  0000                     _SSPCON1	set	4038
    45  0000                     _SSPCON1bits	set	4038
    46  0000                     _SSPSTAT	set	4039
    47  0000                     _SSPSTATbits	set	4039
    48  0000                     _TRISAbits	set	3986
    49  0000                     _TRISB	set	3987
    50  0000                     _TRISBbits	set	3987
    51  0000                     _TRISCbits	set	3988
    52  0000                     _TRISD	set	3989
    53  0000                     _TRISDbits	set	3989
    54                           
    55                           ; #config settings
    56  0000                     
    57                           	psect	cinit
    58  007D96                     __pcinit:
    59                           	opt stack 0
    60  007D96                     start_initialization:
    61                           	opt stack 0
    62  007D96                     __initialization:
    63                           	opt stack 0
    64                           
    65                           ; Initialize objects allocated to COMRAM (5 bytes)
    66                           ; load TBLPTR registers with __pidataCOMRAM
    67  007D96  0EBD               	movlw	low __pidataCOMRAM
    68  007D98  6EF6               	movwf	tblptrl,c
    69  007D9A  0E7C               	movlw	high __pidataCOMRAM
    70  007D9C  6EF7               	movwf	tblptrh,c
    71  007D9E  0E00               	movlw	low (__pidataCOMRAM shr (0+16))
    72  007DA0  6EF8               	movwf	tblptru,c
    73  007DA2  EE00  F02A         	lfsr	0,__pdataCOMRAM
    74  007DA6  EE10 F005          	lfsr	1,5
    75  007DAA                     copy_data0:
    76  007DAA  0009               	tblrd		*+
    77  007DAC  CFF5 FFEE          	movff	tablat,postinc0
    78  007DB0  50E5               	movf	postdec1,w,c
    79  007DB2  50E1               	movf	fsr1l,w,c
    80  007DB4  E1FA               	bnz	copy_data0
    81  007DB6                     end_of_initialization:
    82                           	opt stack 0
    83  007DB6                     __end_of__initialization:
    84                           	opt stack 0
    85  007DB6  0E00               	movlw	low (__Lmediumconst shr (0+16))
    86  007DB8  6EF8               	movwf	tblptru,c
    87  007DBA  0100               	movlb	0
    88  007DBC  EF54  F03F         	goto	_main	;jump to C main() function
    89                           tblptru	equ	0xFF8
    90                           tblptrh	equ	0xFF7
    91                           tblptrl	equ	0xFF6
    92                           tablat	equ	0xFF5
    93                           postinc0	equ	0xFEE
    94                           postdec1	equ	0xFE5
    95                           fsr1l	equ	0xFE1
    96                           
    97                           	psect	dataCOMRAM
    98  00002A                     __pdataCOMRAM:
    99                           	opt stack 0
   100  00002A                     _ADDRESS_DATA_PIPE0:
   101                           	opt stack 0
   102  00002A                     	ds	5
   103                           tblptru	equ	0xFF8
   104                           tblptrh	equ	0xFF7
   105                           tblptrl	equ	0xFF6
   106                           tablat	equ	0xFF5
   107                           postinc0	equ	0xFEE
   108                           postdec1	equ	0xFE5
   109                           fsr1l	equ	0xFE1
   110                           
   111                           	psect	cstackCOMRAM
   112  000001                     __pcstackCOMRAM:
   113                           	opt stack 0
   114  000001                     OpenSPI@bus_mode:
   115                           	opt stack 0
   116  000001                     ReadSPI@TempVar:
   117                           	opt stack 0
   118  000001                     WriteSPI@TempVar:
   119                           	opt stack 0
   120  000001                     Delay_ms@count:
   121                           	opt stack 0
   122                           
   123                           ; 2 bytes @ 0x0
   124  000001                     	ds	1
   125  000002                     OpenSPI@smp_phase:
   126                           	opt stack 0
   127  000002                     WriteSPI@data_out:
   128                           	opt stack 0
   129                           
   130                           ; 1 bytes @ 0x1
   131  000002                     	ds	1
   132  000003                     ??_Delay_ms:
   133  000003                     NRF24L01_WriteRegister@value:
   134                           	opt stack 0
   135  000003                     NRF24L01_ReadRegister@Mnemonic:
   136                           	opt stack 0
   137  000003                     OpenSPI@sync_mode:
   138                           	opt stack 0
   139  000003                     NRF24L01_WriteBuffer@buffer:
   140                           	opt stack 0
   141  000003                     NRF24L01_ReadBuffer@buffer:
   142                           	opt stack 0
   143                           
   144                           ; 2 bytes @ 0x2
   145  000003                     	ds	1
   146  000004                     NRF24L01_WriteRegister@Mnemonic:
   147                           	opt stack 0
   148  000004                     NRF24L01_ReadRegister@byte0:
   149                           	opt stack 0
   150  000004                     Delay_ms@i:
   151                           	opt stack 0
   152                           
   153                           ; 2 bytes @ 0x3
   154  000004                     	ds	1
   155  000005                     ??_NRF24L01_DataReady:
   156  000005                     NRF24L01_WriteBuffer@bytes:
   157                           	opt stack 0
   158  000005                     NRF24L01_ReadBuffer@bytes:
   159                           	opt stack 0
   160  000005                     NRF24L01_SetMode@mode:
   161                           	opt stack 0
   162  000005                     NRF24L01_SetChannel@rf_channel:
   163                           	opt stack 0
   164                           
   165                           ; 1 bytes @ 0x4
   166  000005                     	ds	1
   167  000006                     NRF24L01_WriteBuffer@data:
   168                           	opt stack 0
   169  000006                     NRF24L01_ReadBuffer@data:
   170                           	opt stack 0
   171                           
   172                           ; 1 bytes @ 0x5
   173  000006                     	ds	1
   174  000007                     NRF24L01_WriteBuffer@i:
   175                           	opt stack 0
   176  000007                     NRF24L01_ReadBuffer@i:
   177                           	opt stack 0
   178                           
   179                           ; 1 bytes @ 0x6
   180  000007                     	ds	1
   181  000008                     NRF24L01_Init@rf_channel:
   182                           	opt stack 0
   183  000008                     NRF24L01_ReadData@buffer:
   184                           	opt stack 0
   185                           
   186                           ; 2 bytes @ 0x7
   187  000008                     	ds	1
   188  000009                     NRF24L01_Init@mode:
   189                           	opt stack 0
   190                           
   191                           ; 1 bytes @ 0x8
   192  000009                     	ds	1
   193  00000A                     main@bufferRX:
   194                           	opt stack 0
   195                           
   196                           ; 32 bytes @ 0x9
   197  00000A                     	ds	32
   198                           tblptru	equ	0xFF8
   199                           tblptrh	equ	0xFF7
   200                           tblptrl	equ	0xFF6
   201                           tablat	equ	0xFF5
   202                           postinc0	equ	0xFEE
   203                           postdec1	equ	0xFE5
   204                           fsr1l	equ	0xFE1
   205                           
   206 ;;
   207 ;;Main: autosize = 0, tempsize = 0, incstack = 0, save=0
   208 ;;
   209 ;; *************** function _main *****************
   210 ;; Defined at:
   211 ;;		line 17 in file "RXmain.c"
   212 ;; Parameters:    Size  Location     Type
   213 ;;		None
   214 ;; Auto vars:     Size  Location     Type
   215 ;;  bufferRX       32    9[COMRAM] unsigned char [32]
   216 ;; Return value:  Size  Location     Type
   217 ;;		None               void
   218 ;; Registers used:
   219 ;;		wreg, fsr2l, fsr2h, status,2, status,0, cstack
   220 ;; Tracked objects:
   221 ;;		On entry : 0/0
   222 ;;		On exit  : 0/0
   223 ;;		Unchanged: 0/0
   224 ;; Data sizes:     COMRAM   BANK0   BANK1   BANK2   BANK3   BANK4   BANK5   BANK6   BANK7
   225 ;;      Params:         0       0       0       0       0       0       0       0       0
   226 ;;      Locals:        32       0       0       0       0       0       0       0       0
   227 ;;      Temps:          0       0       0       0       0       0       0       0       0
   228 ;;      Totals:        32       0       0       0       0       0       0       0       0
   229 ;;Total ram usage:       32 bytes
   230 ;; Hardware stack levels required when called:    4
   231 ;; This function calls:
   232 ;;		_NRF24L01_DataReady
   233 ;;		_NRF24L01_Init
   234 ;;		_NRF24L01_ReadData
   235 ;;		_OpenSPI
   236 ;; This function is called by:
   237 ;;		Startup code after reset
   238 ;; This function uses a non-reentrant model
   239 ;;
   240                           
   241                           	psect	text0
   242  007EA8                     __ptext0:
   243                           	opt stack 0
   244  007EA8                     _main:
   245                           	opt stack 27
   246                           
   247                           ;RXmain.c: 18: unsigned char bufferRX[32];
   248                           ;RXmain.c: 19: ADCON0=0x00;
   249                           
   250                           ;incstack = 0
   251  007EA8  0E00               	movlw	0
   252  007EAA  6EC2               	movwf	4034,c	;volatile
   253                           
   254                           ;RXmain.c: 20: ADCON1=0x00;
   255  007EAC  0E00               	movlw	0
   256  007EAE  6EC1               	movwf	4033,c	;volatile
   257                           
   258                           ;RXmain.c: 21: ADCON1bits.PCFG=0x0F;
   259  007EB0  80C1               	bsf	4033,0,c	;volatile
   260  007EB2  82C1               	bsf	4033,1,c	;volatile
   261  007EB4  84C1               	bsf	4033,2,c	;volatile
   262  007EB6  86C1               	bsf	4033,3,c	;volatile
   263                           
   264                           ;RXmain.c: 23: TRISB = 0x00;
   265  007EB8  0E00               	movlw	0
   266  007EBA  6E93               	movwf	3987,c	;volatile
   267                           
   268                           ;RXmain.c: 24: TRISD = 0x00;
   269  007EBC  0E00               	movlw	0
   270  007EBE  6E95               	movwf	3989,c	;volatile
   271                           
   272                           ;RXmain.c: 32: (SSPCON1 &=0xDF);
   273  007EC0  9AC6               	bcf	4038,5,c	;volatile
   274                           
   275                           ;RXmain.c: 33: OpenSPI(0b00000010, 0b00000000, 0b10000000);
   276  007EC2  0E00               	movlw	0
   277  007EC4  6E01               	movwf	OpenSPI@bus_mode,c
   278  007EC6  0E80               	movlw	128
   279  007EC8  6E02               	movwf	OpenSPI@smp_phase,c
   280  007ECA  0E02               	movlw	2
   281  007ECC  EC7C  F03F         	call	_OpenSPI
   282                           
   283                           ;RXmain.c: 35: NRF24L01_Init(1, 0x40);
   284  007ED0  0E40               	movlw	64
   285  007ED2  6E08               	movwf	NRF24L01_Init@rf_channel,c
   286  007ED4  0E01               	movlw	1
   287  007ED6  ECA7  F03F         	call	_NRF24L01_Init
   288  007EDA                     l1377:
   289  007EDA  EC71  F03E         	call	_NRF24L01_DataReady	;wreg free
   290  007EDE  0900               	iorlw	0
   291  007EE0  A4D8               	btfss	status,2,c
   292  007EE2  D7FB               	goto	l1377
   293                           
   294                           ;RXmain.c: 38: NRF24L01_ReadData(bufferRX);
   295  007EE4  0E0A               	movlw	low main@bufferRX
   296  007EE6  6E08               	movwf	NRF24L01_ReadData@buffer,c
   297  007EE8  0E00               	movlw	high main@bufferRX
   298  007EEA  6E09               	movwf	NRF24L01_ReadData@buffer+1,c
   299  007EEC  ECBA  F03E         	call	_NRF24L01_ReadData	;wreg free
   300                           
   301                           ;RXmain.c: 39: LATB = bufferRX[0];
   302  007EF0  C00A  FF8A         	movff	main@bufferRX,3978	;volatile
   303  007EF4  D7F2               	goto	l1377
   304  007EF6  D7FF               	goto	l219
   305  007EF8                     __end_of_main:
   306                           	opt stack 0
   307                           tblptru	equ	0xFF8
   308                           tblptrh	equ	0xFF7
   309                           tblptrl	equ	0xFF6
   310                           tablat	equ	0xFF5
   311                           postinc0	equ	0xFEE
   312                           postdec1	equ	0xFE5
   313                           fsr1l	equ	0xFE1
   314                           status	equ	0xFD8
   315                           
   316 ;; *************** function _OpenSPI *****************
   317 ;; Defined at:
   318 ;;		line 14 in file "C:\Program Files\Microchip\xc8\v1.35\sources\pic18\plib\SPI\spi_open.c"
   319 ;; Parameters:    Size  Location     Type
   320 ;;  sync_mode       1    wreg     unsigned char 
   321 ;;  bus_mode        1    0[COMRAM] unsigned char 
   322 ;;  smp_phase       1    1[COMRAM] unsigned char 
   323 ;; Auto vars:     Size  Location     Type
   324 ;;  sync_mode       1    2[COMRAM] unsigned char 
   325 ;; Return value:  Size  Location     Type
   326 ;;		None               void
   327 ;; Registers used:
   328 ;;		wreg, status,2, status,0
   329 ;; Tracked objects:
   330 ;;		On entry : 0/0
   331 ;;		On exit  : 0/0
   332 ;;		Unchanged: 0/0
   333 ;; Data sizes:     COMRAM   BANK0   BANK1   BANK2   BANK3   BANK4   BANK5   BANK6   BANK7
   334 ;;      Params:         2       0       0       0       0       0       0       0       0
   335 ;;      Locals:         1       0       0       0       0       0       0       0       0
   336 ;;      Temps:          0       0       0       0       0       0       0       0       0
   337 ;;      Totals:         3       0       0       0       0       0       0       0       0
   338 ;;Total ram usage:        3 bytes
   339 ;; Hardware stack levels used:    1
   340 ;; This function calls:
   341 ;;		Nothing
   342 ;; This function is called by:
   343 ;;		_main
   344 ;; This function uses a non-reentrant model
   345 ;;
   346                           
   347                           	psect	text1
   348  007EF8                     __ptext1:
   349                           	opt stack 0
   350  007EF8                     _OpenSPI:
   351                           	opt stack 30
   352                           
   353                           ;incstack = 0
   354                           ;OpenSPI@sync_mode stored from wreg
   355  007EF8  6E03               	movwf	OpenSPI@sync_mode,c
   356  007EFA  0E3F               	movlw	63
   357  007EFC  16C7               	andwf	4039,f,c	;volatile
   358  007EFE  0E00               	movlw	0
   359  007F00  6EC6               	movwf	4038,c	;volatile
   360  007F02  5003               	movf	OpenSPI@sync_mode,w,c
   361  007F04  12C6               	iorwf	4038,f,c	;volatile
   362  007F06  5002               	movf	OpenSPI@smp_phase,w,c
   363  007F08  12C7               	iorwf	4039,f,c	;volatile
   364  007F0A  D005               	goto	l1347
   365  007F0C                     l239:
   366  007F0C  8CC7               	bsf	4039,6,c	;volatile
   367  007F0E  D013               	goto	l1351
   368  007F10                     l241:
   369  007F10  8CC7               	bsf	4039,6,c	;volatile
   370  007F12                     l242:
   371  007F12  88C6               	bsf	4038,4,c	;volatile
   372  007F14  D010               	goto	l1351
   373  007F16                     l1347:
   374  007F16  5001               	movf	OpenSPI@bus_mode,w,c
   375                           
   376                           ; Switch size 1, requested type "space"
   377                           ; Number of cases is 3, Range of values is 0 to 3
   378                           ; switch strategies available:
   379                           ; Name         Instructions Cycles
   380                           ; simple_byte           10     6 (average)
   381                           ;	Chosen strategy is simple_byte
   382  007F18  0A00               	xorlw	0	; case 0
   383  007F1A  B4D8               	btfsc	status,2,c
   384  007F1C  D7F7               	goto	l239
   385  007F1E  0A02               	xorlw	2	; case 2
   386  007F20  B4D8               	btfsc	status,2,c
   387  007F22  D7F6               	goto	l241
   388  007F24  0A01               	xorlw	1	; case 3
   389  007F26  B4D8               	btfsc	status,2,c
   390  007F28  D7F4               	goto	l242
   391  007F2A  D005               	goto	l1351
   392  007F2C                     l245:
   393  007F2C  8A92               	bsf	3986,5,c	;volatile
   394  007F2E                     l247:
   395  007F2E  8293               	bsf	3987,1,c	;volatile
   396  007F30  D00A               	goto	l246
   397  007F32                     l248:
   398  007F32  9293               	bcf	3987,1,c	;volatile
   399  007F34  D008               	goto	l246
   400  007F36                     l1351:
   401  007F36  5003               	movf	OpenSPI@sync_mode,w,c
   402                           
   403                           ; Switch size 1, requested type "space"
   404                           ; Number of cases is 2, Range of values is 4 to 5
   405                           ; switch strategies available:
   406                           ; Name         Instructions Cycles
   407                           ; simple_byte            7     4 (average)
   408                           ;	Chosen strategy is simple_byte
   409  007F38  0A04               	xorlw	4	; case 4
   410  007F3A  B4D8               	btfsc	status,2,c
   411  007F3C  D7F7               	goto	l245
   412  007F3E  0A01               	xorlw	1	; case 5
   413  007F40  B4D8               	btfsc	status,2,c
   414  007F42  D7F5               	goto	l247
   415  007F44  D7F6               	goto	l248
   416  007F46                     l246:
   417  007F46  8093               	bsf	3987,0,c	;volatile
   418  007F48  9E94               	bcf	3988,7,c	;volatile
   419  007F4A  8AC6               	bsf	4038,5,c	;volatile
   420  007F4C  0012               	return		;funcret
   421  007F4E                     __end_of_OpenSPI:
   422                           	opt stack 0
   423                           tblptru	equ	0xFF8
   424                           tblptrh	equ	0xFF7
   425                           tblptrl	equ	0xFF6
   426                           tablat	equ	0xFF5
   427                           postinc0	equ	0xFEE
   428                           postdec1	equ	0xFE5
   429                           fsr1l	equ	0xFE1
   430                           status	equ	0xFD8
   431                           
   432 ;; *************** function _NRF24L01_ReadData *****************
   433 ;; Defined at:
   434 ;;		line 104 in file "nrf24l01.c"
   435 ;; Parameters:    Size  Location     Type
   436 ;;  buffer          2    7[COMRAM] PTR unsigned char 
   437 ;;		 -> main@bufferRX(32), 
   438 ;; Auto vars:     Size  Location     Type
   439 ;;		None
   440 ;; Return value:  Size  Location     Type
   441 ;;		None               void
   442 ;; Registers used:
   443 ;;		wreg, fsr2l, fsr2h, status,2, status,0, cstack
   444 ;; Tracked objects:
   445 ;;		On entry : 0/0
   446 ;;		On exit  : 0/0
   447 ;;		Unchanged: 0/0
   448 ;; Data sizes:     COMRAM   BANK0   BANK1   BANK2   BANK3   BANK4   BANK5   BANK6   BANK7
   449 ;;      Params:         2       0       0       0       0       0       0       0       0
   450 ;;      Locals:         0       0       0       0       0       0       0       0       0
   451 ;;      Temps:          0       0       0       0       0       0       0       0       0
   452 ;;      Totals:         2       0       0       0       0       0       0       0       0
   453 ;;Total ram usage:        2 bytes
   454 ;; Hardware stack levels used:    1
   455 ;; Hardware stack levels required when called:    2
   456 ;; This function calls:
   457 ;;		_NRF24L01_Flush
   458 ;;		_NRF24L01_ReadBuffer
   459 ;;		_NRF24L01_WriteRegister
   460 ;; This function is called by:
   461 ;;		_main
   462 ;; This function uses a non-reentrant model
   463 ;;
   464                           
   465                           	psect	text2
   466  007D74                     __ptext2:
   467                           	opt stack 0
   468  007D74                     _NRF24L01_ReadData:
   469                           	opt stack 28
   470                           
   471                           ;nrf24l01.c: 105: NRF24L01_ReadBuffer(0x61, buffer, 1);
   472                           
   473                           ;incstack = 0
   474  007D74  C008  F003         	movff	NRF24L01_ReadData@buffer,NRF24L01_ReadBuffer@buffer
   475  007D78  C009  F004         	movff	NRF24L01_ReadData@buffer+1,NRF24L01_ReadBuffer@buffer+1
   476  007D7C  0E01               	movlw	1
   477  007D7E  6E05               	movwf	NRF24L01_ReadBuffer@bytes,c
   478  007D80  0E61               	movlw	97
   479  007D82  EC33  F03F         	call	_NRF24L01_ReadBuffer
   480                           
   481                           ;nrf24l01.c: 106: NRF24L01_WriteRegister(0x07, 0x70);
   482  007D86  0E70               	movlw	112
   483  007D88  6E03               	movwf	NRF24L01_WriteRegister@value,c
   484  007D8A  0E07               	movlw	7
   485  007D8C  EC98  F03E         	call	_NRF24L01_WriteRegister
   486                           
   487                           ;nrf24l01.c: 107: NRF24L01_Flush();
   488  007D90  ECA9  F03E         	call	_NRF24L01_Flush	;wreg free
   489  007D94  0012               	return		;funcret
   490  007D96                     __end_of_NRF24L01_ReadData:
   491                           	opt stack 0
   492                           tblptru	equ	0xFF8
   493                           tblptrh	equ	0xFF7
   494                           tblptrl	equ	0xFF6
   495                           tablat	equ	0xFF5
   496                           postinc0	equ	0xFEE
   497                           postdec1	equ	0xFE5
   498                           fsr1l	equ	0xFE1
   499                           status	equ	0xFD8
   500                           
   501 ;; *************** function _NRF24L01_ReadBuffer *****************
   502 ;; Defined at:
   503 ;;		line 43 in file "nrf24l01.c"
   504 ;; Parameters:    Size  Location     Type
   505 ;;  data            1    wreg     unsigned char 
   506 ;;  buffer          2    2[COMRAM] PTR unsigned char 
   507 ;;		 -> main@bufferRX(32), 
   508 ;;  bytes           1    4[COMRAM] unsigned char 
   509 ;; Auto vars:     Size  Location     Type
   510 ;;  data            1    5[COMRAM] unsigned char 
   511 ;;  i               1    6[COMRAM] unsigned char 
   512 ;; Return value:  Size  Location     Type
   513 ;;		None               void
   514 ;; Registers used:
   515 ;;		wreg, fsr2l, fsr2h, status,2, status,0, cstack
   516 ;; Tracked objects:
   517 ;;		On entry : 0/0
   518 ;;		On exit  : 0/0
   519 ;;		Unchanged: 0/0
   520 ;; Data sizes:     COMRAM   BANK0   BANK1   BANK2   BANK3   BANK4   BANK5   BANK6   BANK7
   521 ;;      Params:         3       0       0       0       0       0       0       0       0
   522 ;;      Locals:         2       0       0       0       0       0       0       0       0
   523 ;;      Temps:          0       0       0       0       0       0       0       0       0
   524 ;;      Totals:         5       0       0       0       0       0       0       0       0
   525 ;;Total ram usage:        5 bytes
   526 ;; Hardware stack levels used:    1
   527 ;; Hardware stack levels required when called:    1
   528 ;; This function calls:
   529 ;;		_ReadSPI
   530 ;;		_WriteSPI
   531 ;; This function is called by:
   532 ;;		_NRF24L01_ReadData
   533 ;; This function uses a non-reentrant model
   534 ;;
   535                           
   536                           	psect	text3
   537  007E66                     __ptext3:
   538                           	opt stack 0
   539  007E66                     _NRF24L01_ReadBuffer:
   540                           	opt stack 28
   541                           
   542                           ;incstack = 0
   543                           ;NRF24L01_ReadBuffer@data stored from wreg
   544  007E66  6E06               	movwf	NRF24L01_ReadBuffer@data,c
   545                           
   546                           ;nrf24l01.c: 44: unsigned char i;
   547                           ;nrf24l01.c: 45: LATDbits.LATD1 = 0;
   548  007E68  928C               	bcf	3980,1,c	;volatile
   549  007E6A                     l1289:
   550  007E6A  5006               	movf	NRF24L01_ReadBuffer@data,w,c
   551  007E6C  EC89  F03E         	call	_WriteSPI
   552  007E70  0900               	iorlw	0
   553  007E72  A4D8               	btfss	status,2,c
   554  007E74  D7FA               	goto	l1289
   555                           
   556                           ;nrf24l01.c: 47: for(i = 0; i < bytes; i++){
   557  007E76  0E00               	movlw	0
   558  007E78  6E07               	movwf	NRF24L01_ReadBuffer@i,c
   559  007E7A  D00A               	goto	l1299
   560  007E7C                     l1293:
   561                           
   562                           ;nrf24l01.c: 48: *buffer = ReadSPI();
   563  007E7C  EC68  F03E         	call	_ReadSPI	;wreg free
   564  007E80  C003  FFD9         	movff	NRF24L01_ReadBuffer@buffer,fsr2l
   565  007E84  C004  FFDA         	movff	NRF24L01_ReadBuffer@buffer+1,fsr2h
   566  007E88  6EDF               	movwf	indf2,c
   567                           
   568                           ;nrf24l01.c: 49: buffer++;
   569  007E8A  4A03               	infsnz	NRF24L01_ReadBuffer@buffer,f,c
   570  007E8C  2A04               	incf	NRF24L01_ReadBuffer@buffer+1,f,c
   571  007E8E  2A07               	incf	NRF24L01_ReadBuffer@i,f,c
   572  007E90                     l1299:
   573  007E90  5005               	movf	NRF24L01_ReadBuffer@bytes,w,c
   574  007E92  5C07               	subwf	NRF24L01_ReadBuffer@i,w,c
   575  007E94  A0D8               	btfss	status,0,c
   576  007E96  D7F2               	goto	l1293
   577                           
   578                           ;nrf24l01.c: 50: }
   579                           ;nrf24l01.c: 51: *buffer = (0);
   580  007E98  C003  FFD9         	movff	NRF24L01_ReadBuffer@buffer,fsr2l
   581  007E9C  C004  FFDA         	movff	NRF24L01_ReadBuffer@buffer+1,fsr2h
   582  007EA0  0E00               	movlw	0
   583  007EA2  6EDF               	movwf	indf2,c
   584                           
   585                           ;nrf24l01.c: 52: LATDbits.LATD1 = 1;
   586  007EA4  828C               	bsf	3980,1,c	;volatile
   587  007EA6  0012               	return		;funcret
   588  007EA8                     __end_of_NRF24L01_ReadBuffer:
   589                           	opt stack 0
   590                           tblptru	equ	0xFF8
   591                           tblptrh	equ	0xFF7
   592                           tblptrl	equ	0xFF6
   593                           tablat	equ	0xFF5
   594                           postinc0	equ	0xFEE
   595                           postdec1	equ	0xFE5
   596                           fsr1l	equ	0xFE1
   597                           indf2	equ	0xFDF
   598                           fsr2h	equ	0xFDA
   599                           fsr2l	equ	0xFD9
   600                           status	equ	0xFD8
   601                           
   602 ;; *************** function _NRF24L01_Init *****************
   603 ;; Defined at:
   604 ;;		line 55 in file "nrf24l01.c"
   605 ;; Parameters:    Size  Location     Type
   606 ;;  mode            1    wreg     unsigned char 
   607 ;;  rf_channel      1    7[COMRAM] unsigned char 
   608 ;; Auto vars:     Size  Location     Type
   609 ;;  mode            1    8[COMRAM] unsigned char 
   610 ;; Return value:  Size  Location     Type
   611 ;;		None               void
   612 ;; Registers used:
   613 ;;		wreg, fsr2l, fsr2h, status,2, status,0, cstack
   614 ;; Tracked objects:
   615 ;;		On entry : 0/0
   616 ;;		On exit  : 0/0
   617 ;;		Unchanged: 0/0
   618 ;; Data sizes:     COMRAM   BANK0   BANK1   BANK2   BANK3   BANK4   BANK5   BANK6   BANK7
   619 ;;      Params:         1       0       0       0       0       0       0       0       0
   620 ;;      Locals:         1       0       0       0       0       0       0       0       0
   621 ;;      Temps:          0       0       0       0       0       0       0       0       0
   622 ;;      Totals:         2       0       0       0       0       0       0       0       0
   623 ;;Total ram usage:        2 bytes
   624 ;; Hardware stack levels used:    1
   625 ;; Hardware stack levels required when called:    3
   626 ;; This function calls:
   627 ;;		_Delay_ms
   628 ;;		_NRF24L01_SetChannel
   629 ;;		_NRF24L01_SetMode
   630 ;;		_NRF24L01_WriteBuffer
   631 ;;		_NRF24L01_WriteRegister
   632 ;; This function is called by:
   633 ;;		_main
   634 ;; This function uses a non-reentrant model
   635 ;;
   636                           
   637                           	psect	text4
   638  007F4E                     __ptext4:
   639                           	opt stack 0
   640  007F4E                     _NRF24L01_Init:
   641                           	opt stack 27
   642                           
   643                           ;incstack = 0
   644                           ;NRF24L01_Init@mode stored from wreg
   645  007F4E  6E09               	movwf	NRF24L01_Init@mode,c
   646                           
   647                           ;nrf24l01.c: 56: TRISDbits.TRISD1 = 0; TRISDbits.TRISD0 = 0;
   648  007F50  9295               	bcf	3989,1,c	;volatile
   649  007F52  9095               	bcf	3989,0,c	;volatile
   650                           
   651                           ;nrf24l01.c: 57: LATDbits.LATD1 = 1; LATDbits.LATD0 = 0;
   652  007F54  828C               	bsf	3980,1,c	;volatile
   653  007F56  908C               	bcf	3980,0,c	;volatile
   654                           
   655                           ;nrf24l01.c: 58: Delay_ms(100);
   656  007F58  0E00               	movlw	0
   657  007F5A  6E02               	movwf	Delay_ms@count+1,c
   658  007F5C  0E64               	movlw	100
   659  007F5E  6E01               	movwf	Delay_ms@count,c
   660  007F60  ECE0  F03E         	call	_Delay_ms	;wreg free
   661                           
   662                           ;nrf24l01.c: 59: NRF24L01_WriteRegister(0x00, 0x0A); Delay_ms(10);
   663  007F64  0E0A               	movlw	10
   664  007F66  6E03               	movwf	NRF24L01_WriteRegister@value,c
   665  007F68  0E00               	movlw	0
   666  007F6A  EC98  F03E         	call	_NRF24L01_WriteRegister
   667  007F6E  0E00               	movlw	0
   668  007F70  6E02               	movwf	Delay_ms@count+1,c
   669  007F72  0E0A               	movlw	10
   670  007F74  6E01               	movwf	Delay_ms@count,c
   671  007F76  ECE0  F03E         	call	_Delay_ms	;wreg free
   672                           
   673                           ;nrf24l01.c: 60: NRF24L01_WriteRegister(0x01, 0x01);
   674  007F7A  0E01               	movlw	1
   675  007F7C  6E03               	movwf	NRF24L01_WriteRegister@value,c
   676  007F7E  0E01               	movlw	1
   677  007F80  EC98  F03E         	call	_NRF24L01_WriteRegister
   678                           
   679                           ;nrf24l01.c: 61: NRF24L01_WriteRegister(0x02, 0x01);
   680  007F84  0E01               	movlw	1
   681  007F86  6E03               	movwf	NRF24L01_WriteRegister@value,c
   682  007F88  0E02               	movlw	2
   683  007F8A  EC98  F03E         	call	_NRF24L01_WriteRegister
   684                           
   685                           ;nrf24l01.c: 62: NRF24L01_WriteRegister(0x03, 0x03);
   686  007F8E  0E03               	movlw	3
   687  007F90  6E03               	movwf	NRF24L01_WriteRegister@value,c
   688  007F92  0E03               	movlw	3
   689  007F94  EC98  F03E         	call	_NRF24L01_WriteRegister
   690                           
   691                           ;nrf24l01.c: 63: NRF24L01_WriteRegister(0x04, 0x00);
   692  007F98  0E00               	movlw	0
   693  007F9A  6E03               	movwf	NRF24L01_WriteRegister@value,c
   694  007F9C  0E04               	movlw	4
   695  007F9E  EC98  F03E         	call	_NRF24L01_WriteRegister
   696                           
   697                           ;nrf24l01.c: 64: NRF24L01_SetChannel(rf_channel);
   698  007FA2  5008               	movf	NRF24L01_Init@rf_channel,w,c
   699  007FA4  EC61  F03E         	call	_NRF24L01_SetChannel
   700                           
   701                           ;nrf24l01.c: 65: NRF24L01_WriteRegister(0x06, 0x0E);
   702  007FA8  0E0E               	movlw	14
   703  007FAA  6E03               	movwf	NRF24L01_WriteRegister@value,c
   704  007FAC  0E06               	movlw	6
   705  007FAE  EC98  F03E         	call	_NRF24L01_WriteRegister
   706                           
   707                           ;nrf24l01.c: 67: NRF24L01_WriteBuffer(0x20 | 0x0A, ADDRESS_DATA_PIPE0, 5);
   708  007FB2  0E2A               	movlw	low _ADDRESS_DATA_PIPE0
   709  007FB4  6E03               	movwf	NRF24L01_WriteBuffer@buffer,c
   710  007FB6  0E00               	movlw	high _ADDRESS_DATA_PIPE0
   711  007FB8  6E04               	movwf	NRF24L01_WriteBuffer@buffer+1,c
   712  007FBA  0E05               	movlw	5
   713  007FBC  6E05               	movwf	NRF24L01_WriteBuffer@bytes,c
   714  007FBE  0E2A               	movlw	42
   715  007FC0  ECF6  F03E         	call	_NRF24L01_WriteBuffer
   716                           
   717                           ;nrf24l01.c: 68: NRF24L01_WriteBuffer(0x20 | 0x10, ADDRESS_DATA_PIPE0, 5);
   718  007FC4  0E2A               	movlw	low _ADDRESS_DATA_PIPE0
   719  007FC6  6E03               	movwf	NRF24L01_WriteBuffer@buffer,c
   720  007FC8  0E00               	movlw	high _ADDRESS_DATA_PIPE0
   721  007FCA  6E04               	movwf	NRF24L01_WriteBuffer@buffer+1,c
   722  007FCC  0E05               	movlw	5
   723  007FCE  6E05               	movwf	NRF24L01_WriteBuffer@bytes,c
   724  007FD0  0E30               	movlw	48
   725  007FD2  ECF6  F03E         	call	_NRF24L01_WriteBuffer
   726                           
   727                           ;nrf24l01.c: 69: NRF24L01_WriteRegister(0x11, 1);
   728  007FD6  0E01               	movlw	1
   729  007FD8  6E03               	movwf	NRF24L01_WriteRegister@value,c
   730  007FDA  0E11               	movlw	17
   731  007FDC  EC98  F03E         	call	_NRF24L01_WriteRegister
   732                           
   733                           ;nrf24l01.c: 71: Delay_ms(100);
   734  007FE0  0E00               	movlw	0
   735  007FE2  6E02               	movwf	Delay_ms@count+1,c
   736  007FE4  0E64               	movlw	100
   737  007FE6  6E01               	movwf	Delay_ms@count,c
   738  007FE8  ECE0  F03E         	call	_Delay_ms	;wreg free
   739                           
   740                           ;nrf24l01.c: 72: NRF24L01_SetMode(mode);
   741  007FEC  5009               	movf	NRF24L01_Init@mode,w,c
   742  007FEE  EC14  F03F         	call	_NRF24L01_SetMode
   743                           
   744                           ;nrf24l01.c: 73: Delay_ms(100);
   745  007FF2  0E00               	movlw	0
   746  007FF4  6E02               	movwf	Delay_ms@count+1,c
   747  007FF6  0E64               	movlw	100
   748  007FF8  6E01               	movwf	Delay_ms@count,c
   749  007FFA  ECE0  F03E         	call	_Delay_ms	;wreg free
   750  007FFE  0012               	return		;funcret
   751  008000                     __end_of_NRF24L01_Init:
   752                           	opt stack 0
   753                           tblptru	equ	0xFF8
   754                           tblptrh	equ	0xFF7
   755                           tblptrl	equ	0xFF6
   756                           tablat	equ	0xFF5
   757                           postinc0	equ	0xFEE
   758                           postdec1	equ	0xFE5
   759                           fsr1l	equ	0xFE1
   760                           indf2	equ	0xFDF
   761                           fsr2h	equ	0xFDA
   762                           fsr2l	equ	0xFD9
   763                           status	equ	0xFD8
   764                           
   765 ;; *************** function _NRF24L01_WriteBuffer *****************
   766 ;; Defined at:
   767 ;;		line 32 in file "nrf24l01.c"
   768 ;; Parameters:    Size  Location     Type
   769 ;;  data            1    wreg     unsigned char 
   770 ;;  buffer          2    2[COMRAM] PTR unsigned char 
   771 ;;		 -> ADDRESS_DATA_PIPE0(5), 
   772 ;;  bytes           1    4[COMRAM] unsigned char 
   773 ;; Auto vars:     Size  Location     Type
   774 ;;  data            1    5[COMRAM] unsigned char 
   775 ;;  i               1    6[COMRAM] unsigned char 
   776 ;; Return value:  Size  Location     Type
   777 ;;		None               void
   778 ;; Registers used:
   779 ;;		wreg, fsr2l, fsr2h, status,2, status,0, cstack
   780 ;; Tracked objects:
   781 ;;		On entry : 0/0
   782 ;;		On exit  : 0/0
   783 ;;		Unchanged: 0/0
   784 ;; Data sizes:     COMRAM   BANK0   BANK1   BANK2   BANK3   BANK4   BANK5   BANK6   BANK7
   785 ;;      Params:         3       0       0       0       0       0       0       0       0
   786 ;;      Locals:         2       0       0       0       0       0       0       0       0
   787 ;;      Temps:          0       0       0       0       0       0       0       0       0
   788 ;;      Totals:         5       0       0       0       0       0       0       0       0
   789 ;;Total ram usage:        5 bytes
   790 ;; Hardware stack levels used:    1
   791 ;; Hardware stack levels required when called:    1
   792 ;; This function calls:
   793 ;;		_WriteSPI
   794 ;; This function is called by:
   795 ;;		_NRF24L01_Init
   796 ;;		_NRF24L01_SendData
   797 ;; This function uses a non-reentrant model
   798 ;;
   799                           
   800                           	psect	text5
   801  007DEC                     __ptext5:
   802                           	opt stack 0
   803  007DEC                     _NRF24L01_WriteBuffer:
   804                           	opt stack 28
   805                           
   806                           ;incstack = 0
   807                           ;NRF24L01_WriteBuffer@data stored from wreg
   808  007DEC  6E06               	movwf	NRF24L01_WriteBuffer@data,c
   809                           
   810                           ;nrf24l01.c: 33: unsigned char i;
   811                           ;nrf24l01.c: 34: LATDbits.LATD1 = 0;
   812  007DEE  928C               	bcf	3980,1,c	;volatile
   813  007DF0                     l1277:
   814  007DF0  5006               	movf	NRF24L01_WriteBuffer@data,w,c
   815  007DF2  EC89  F03E         	call	_WriteSPI
   816  007DF6  0900               	iorlw	0
   817  007DF8  A4D8               	btfss	status,2,c
   818  007DFA  D7FA               	goto	l1277
   819                           
   820                           ;nrf24l01.c: 36: for(i = 0; i < bytes; i++){
   821  007DFC  0E00               	movlw	0
   822  007DFE  6E07               	movwf	NRF24L01_WriteBuffer@i,c
   823  007E00  D00D               	goto	l1285
   824  007E02                     l1281:
   825  007E02  C003  FFD9         	movff	NRF24L01_WriteBuffer@buffer,fsr2l
   826  007E06  C004  FFDA         	movff	NRF24L01_WriteBuffer@buffer+1,fsr2h
   827  007E0A  50DF               	movf	indf2,w,c
   828  007E0C  EC89  F03E         	call	_WriteSPI
   829  007E10  0900               	iorlw	0
   830  007E12  A4D8               	btfss	status,2,c
   831  007E14  D7F6               	goto	l1281
   832                           
   833                           ;nrf24l01.c: 38: buffer++;
   834  007E16  4A03               	infsnz	NRF24L01_WriteBuffer@buffer,f,c
   835  007E18  2A04               	incf	NRF24L01_WriteBuffer@buffer+1,f,c
   836  007E1A  2A07               	incf	NRF24L01_WriteBuffer@i,f,c
   837  007E1C                     l1285:
   838  007E1C  5005               	movf	NRF24L01_WriteBuffer@bytes,w,c
   839  007E1E  5C07               	subwf	NRF24L01_WriteBuffer@i,w,c
   840  007E20  A0D8               	btfss	status,0,c
   841  007E22  D7EF               	goto	l1281
   842                           
   843                           ;nrf24l01.c: 39: }
   844                           ;nrf24l01.c: 40: LATDbits.LATD1 = 1;
   845  007E24  828C               	bsf	3980,1,c	;volatile
   846  007E26  0012               	return		;funcret
   847  007E28                     __end_of_NRF24L01_WriteBuffer:
   848                           	opt stack 0
   849                           tblptru	equ	0xFF8
   850                           tblptrh	equ	0xFF7
   851                           tblptrl	equ	0xFF6
   852                           tablat	equ	0xFF5
   853                           postinc0	equ	0xFEE
   854                           postdec1	equ	0xFE5
   855                           fsr1l	equ	0xFE1
   856                           indf2	equ	0xFDF
   857                           fsr2h	equ	0xFDA
   858                           fsr2l	equ	0xFD9
   859                           status	equ	0xFD8
   860                           
   861 ;; *************** function _NRF24L01_SetMode *****************
   862 ;; Defined at:
   863 ;;		line 76 in file "nrf24l01.c"
   864 ;; Parameters:    Size  Location     Type
   865 ;;  mode            1    wreg     unsigned char 
   866 ;; Auto vars:     Size  Location     Type
   867 ;;  mode            1    4[COMRAM] unsigned char 
   868 ;; Return value:  Size  Location     Type
   869 ;;		None               void
   870 ;; Registers used:
   871 ;;		wreg, status,2, status,0, cstack
   872 ;; Tracked objects:
   873 ;;		On entry : 0/0
   874 ;;		On exit  : 0/0
   875 ;;		Unchanged: 0/0
   876 ;; Data sizes:     COMRAM   BANK0   BANK1   BANK2   BANK3   BANK4   BANK5   BANK6   BANK7
   877 ;;      Params:         0       0       0       0       0       0       0       0       0
   878 ;;      Locals:         1       0       0       0       0       0       0       0       0
   879 ;;      Temps:          0       0       0       0       0       0       0       0       0
   880 ;;      Totals:         1       0       0       0       0       0       0       0       0
   881 ;;Total ram usage:        1 bytes
   882 ;; Hardware stack levels used:    1
   883 ;; Hardware stack levels required when called:    2
   884 ;; This function calls:
   885 ;;		_NRF24L01_Flush
   886 ;;		_NRF24L01_WriteRegister
   887 ;; This function is called by:
   888 ;;		_NRF24L01_Init
   889 ;;		_NRF24L01_SendData
   890 ;; This function uses a non-reentrant model
   891 ;;
   892                           
   893                           	psect	text6
   894  007E28                     __ptext6:
   895                           	opt stack 0
   896  007E28                     _NRF24L01_SetMode:
   897                           	opt stack 27
   898                           
   899                           ;incstack = 0
   900                           ;NRF24L01_SetMode@mode stored from wreg
   901  007E28  6E05               	movwf	NRF24L01_SetMode@mode,c
   902                           
   903                           ;nrf24l01.c: 77: NRF24L01_Flush();
   904  007E2A  ECA9  F03E         	call	_NRF24L01_Flush	;wreg free
   905                           
   906                           ;nrf24l01.c: 78: NRF24L01_WriteRegister(0x07, 0x70);
   907  007E2E  0E70               	movlw	112
   908  007E30  6E03               	movwf	NRF24L01_WriteRegister@value,c
   909  007E32  0E07               	movlw	7
   910  007E34  EC98  F03E         	call	_NRF24L01_WriteRegister
   911                           
   912                           ;nrf24l01.c: 79: switch(mode){
   913  007E38  D00E               	goto	l1321
   914  007E3A                     l1311:
   915                           
   916                           ;nrf24l01.c: 81: NRF24L01_WriteRegister(0x00, 0x0F);
   917  007E3A  0E0F               	movlw	15
   918  007E3C  6E03               	movwf	NRF24L01_WriteRegister@value,c
   919  007E3E  0E00               	movlw	0
   920  007E40  EC98  F03E         	call	_NRF24L01_WriteRegister
   921                           
   922                           ;nrf24l01.c: 82: LATDbits.LATD0 = 1;
   923  007E44  808C               	bsf	3980,0,c	;volatile
   924                           
   925                           ;nrf24l01.c: 83: break;
   926  007E46  0012               	return	
   927  007E48                     l1315:
   928                           
   929                           ;nrf24l01.c: 85: NRF24L01_WriteRegister(0x00, 0x0E);
   930  007E48  0E0E               	movlw	14
   931  007E4A  6E03               	movwf	NRF24L01_WriteRegister@value,c
   932  007E4C  0E00               	movlw	0
   933  007E4E  EC98  F03E         	call	_NRF24L01_WriteRegister
   934                           
   935                           ;nrf24l01.c: 86: LATDbits.LATD0 = 0;
   936  007E52  908C               	bcf	3980,0,c	;volatile
   937                           
   938                           ;nrf24l01.c: 88: }
   939                           
   940                           ;nrf24l01.c: 87: break;
   941  007E54  0012               	return	
   942  007E56                     l1321:
   943  007E56  5005               	movf	NRF24L01_SetMode@mode,w,c
   944                           
   945                           ; Switch size 1, requested type "space"
   946                           ; Number of cases is 2, Range of values is 1 to 2
   947                           ; switch strategies available:
   948                           ; Name         Instructions Cycles
   949                           ; simple_byte            7     4 (average)
   950                           ;	Chosen strategy is simple_byte
   951  007E58  0A01               	xorlw	1	; case 1
   952  007E5A  B4D8               	btfsc	status,2,c
   953  007E5C  D7EE               	goto	l1311
   954  007E5E  0A03               	xorlw	3	; case 2
   955  007E60  A4D8               	btfss	status,2,c
   956  007E62  0012               	return	
   957  007E64  D7F1               	goto	l1315
   958  007E66                     __end_of_NRF24L01_SetMode:
   959                           	opt stack 0
   960                           tblptru	equ	0xFF8
   961                           tblptrh	equ	0xFF7
   962                           tblptrl	equ	0xFF6
   963                           tablat	equ	0xFF5
   964                           postinc0	equ	0xFEE
   965                           postdec1	equ	0xFE5
   966                           fsr1l	equ	0xFE1
   967                           indf2	equ	0xFDF
   968                           fsr2h	equ	0xFDA
   969                           fsr2l	equ	0xFD9
   970                           status	equ	0xFD8
   971                           
   972 ;; *************** function _NRF24L01_Flush *****************
   973 ;; Defined at:
   974 ;;		line 123 in file "nrf24l01.c"
   975 ;; Parameters:    Size  Location     Type
   976 ;;		None
   977 ;; Auto vars:     Size  Location     Type
   978 ;;		None
   979 ;; Return value:  Size  Location     Type
   980 ;;		None               void
   981 ;; Registers used:
   982 ;;		wreg, status,2, cstack
   983 ;; Tracked objects:
   984 ;;		On entry : 0/0
   985 ;;		On exit  : 0/0
   986 ;;		Unchanged: 0/0
   987 ;; Data sizes:     COMRAM   BANK0   BANK1   BANK2   BANK3   BANK4   BANK5   BANK6   BANK7
   988 ;;      Params:         0       0       0       0       0       0       0       0       0
   989 ;;      Locals:         0       0       0       0       0       0       0       0       0
   990 ;;      Temps:          0       0       0       0       0       0       0       0       0
   991 ;;      Totals:         0       0       0       0       0       0       0       0       0
   992 ;;Total ram usage:        0 bytes
   993 ;; Hardware stack levels used:    1
   994 ;; Hardware stack levels required when called:    1
   995 ;; This function calls:
   996 ;;		_WriteSPI
   997 ;; This function is called by:
   998 ;;		_NRF24L01_SetMode
   999 ;;		_NRF24L01_ReadData
  1000 ;; This function uses a non-reentrant model
  1001 ;;
  1002                           
  1003                           	psect	text7
  1004  007D52                     __ptext7:
  1005                           	opt stack 0
  1006  007D52                     _NRF24L01_Flush:
  1007                           	opt stack 28
  1008                           
  1009                           ;nrf24l01.c: 124: LATDbits.LATD1 = 0;
  1010                           
  1011                           ;incstack = 0
  1012  007D52  928C               	bcf	3980,1,c	;volatile
  1013  007D54                     l921:
  1014  007D54  0EE1               	movlw	225
  1015  007D56  EC89  F03E         	call	_WriteSPI
  1016  007D5A  0900               	iorlw	0
  1017  007D5C  A4D8               	btfss	status,2,c
  1018  007D5E  D7FA               	goto	l921
  1019                           
  1020                           ;nrf24l01.c: 126: LATDbits.LATD1 = 1;
  1021  007D60  828C               	bsf	3980,1,c	;volatile
  1022                           
  1023                           ;nrf24l01.c: 127: LATDbits.LATD1 = 0;
  1024  007D62  928C               	bcf	3980,1,c	;volatile
  1025  007D64                     l923:
  1026  007D64  0EE2               	movlw	226
  1027  007D66  EC89  F03E         	call	_WriteSPI
  1028  007D6A  0900               	iorlw	0
  1029  007D6C  A4D8               	btfss	status,2,c
  1030  007D6E  D7FA               	goto	l923
  1031                           
  1032                           ;nrf24l01.c: 129: LATDbits.LATD1 = 1;
  1033  007D70  828C               	bsf	3980,1,c	;volatile
  1034  007D72  0012               	return		;funcret
  1035  007D74                     __end_of_NRF24L01_Flush:
  1036                           	opt stack 0
  1037                           tblptru	equ	0xFF8
  1038                           tblptrh	equ	0xFF7
  1039                           tblptrl	equ	0xFF6
  1040                           tablat	equ	0xFF5
  1041                           postinc0	equ	0xFEE
  1042                           postdec1	equ	0xFE5
  1043                           fsr1l	equ	0xFE1
  1044                           indf2	equ	0xFDF
  1045                           fsr2h	equ	0xFDA
  1046                           fsr2l	equ	0xFD9
  1047                           status	equ	0xFD8
  1048                           
  1049 ;; *************** function _NRF24L01_SetChannel *****************
  1050 ;; Defined at:
  1051 ;;		line 110 in file "nrf24l01.c"
  1052 ;; Parameters:    Size  Location     Type
  1053 ;;  rf_channel      1    wreg     unsigned char 
  1054 ;; Auto vars:     Size  Location     Type
  1055 ;;  rf_channel      1    4[COMRAM] unsigned char 
  1056 ;; Return value:  Size  Location     Type
  1057 ;;		None               void
  1058 ;; Registers used:
  1059 ;;		wreg, status,2, status,0, cstack
  1060 ;; Tracked objects:
  1061 ;;		On entry : 0/0
  1062 ;;		On exit  : 0/0
  1063 ;;		Unchanged: 0/0
  1064 ;; Data sizes:     COMRAM   BANK0   BANK1   BANK2   BANK3   BANK4   BANK5   BANK6   BANK7
  1065 ;;      Params:         0       0       0       0       0       0       0       0       0
  1066 ;;      Locals:         1       0       0       0       0       0       0       0       0
  1067 ;;      Temps:          0       0       0       0       0       0       0       0       0
  1068 ;;      Totals:         1       0       0       0       0       0       0       0       0
  1069 ;;Total ram usage:        1 bytes
  1070 ;; Hardware stack levels used:    1
  1071 ;; Hardware stack levels required when called:    2
  1072 ;; This function calls:
  1073 ;;		_NRF24L01_WriteRegister
  1074 ;; This function is called by:
  1075 ;;		_NRF24L01_Init
  1076 ;; This function uses a non-reentrant model
  1077 ;;
  1078                           
  1079                           	psect	text8
  1080  007CC2                     __ptext8:
  1081                           	opt stack 0
  1082  007CC2                     _NRF24L01_SetChannel:
  1083                           	opt stack 27
  1084                           
  1085                           ;incstack = 0
  1086                           ;NRF24L01_SetChannel@rf_channel stored from wreg
  1087  007CC2  6E05               	movwf	NRF24L01_SetChannel@rf_channel,c
  1088                           
  1089                           ;nrf24l01.c: 111: NRF24L01_WriteRegister(0x05, rf_channel);
  1090  007CC4  C005  F003         	movff	NRF24L01_SetChannel@rf_channel,NRF24L01_WriteRegister@value
  1091  007CC8  0E05               	movlw	5
  1092  007CCA  EC98  F03E         	call	_NRF24L01_WriteRegister
  1093  007CCE  0012               	return		;funcret
  1094  007CD0                     __end_of_NRF24L01_SetChannel:
  1095                           	opt stack 0
  1096                           tblptru	equ	0xFF8
  1097                           tblptrh	equ	0xFF7
  1098                           tblptrl	equ	0xFF6
  1099                           tablat	equ	0xFF5
  1100                           postinc0	equ	0xFEE
  1101                           postdec1	equ	0xFE5
  1102                           fsr1l	equ	0xFE1
  1103                           indf2	equ	0xFDF
  1104                           fsr2h	equ	0xFDA
  1105                           fsr2l	equ	0xFD9
  1106                           status	equ	0xFD8
  1107                           
  1108 ;; *************** function _NRF24L01_WriteRegister *****************
  1109 ;; Defined at:
  1110 ;;		line 16 in file "nrf24l01.c"
  1111 ;; Parameters:    Size  Location     Type
  1112 ;;  Mnemonic        1    wreg     unsigned char 
  1113 ;;  value           1    2[COMRAM] unsigned char 
  1114 ;; Auto vars:     Size  Location     Type
  1115 ;;  Mnemonic        1    3[COMRAM] unsigned char 
  1116 ;; Return value:  Size  Location     Type
  1117 ;;		None               void
  1118 ;; Registers used:
  1119 ;;		wreg, status,2, status,0, cstack
  1120 ;; Tracked objects:
  1121 ;;		On entry : 0/0
  1122 ;;		On exit  : 0/0
  1123 ;;		Unchanged: 0/0
  1124 ;; Data sizes:     COMRAM   BANK0   BANK1   BANK2   BANK3   BANK4   BANK5   BANK6   BANK7
  1125 ;;      Params:         1       0       0       0       0       0       0       0       0
  1126 ;;      Locals:         1       0       0       0       0       0       0       0       0
  1127 ;;      Temps:          0       0       0       0       0       0       0       0       0
  1128 ;;      Totals:         2       0       0       0       0       0       0       0       0
  1129 ;;Total ram usage:        2 bytes
  1130 ;; Hardware stack levels used:    1
  1131 ;; Hardware stack levels required when called:    1
  1132 ;; This function calls:
  1133 ;;		_WriteSPI
  1134 ;; This function is called by:
  1135 ;;		_NRF24L01_Init
  1136 ;;		_NRF24L01_SetMode
  1137 ;;		_NRF24L01_ReadData
  1138 ;;		_NRF24L01_SetChannel
  1139 ;;		_NRF24L01_StandbyI
  1140 ;; This function uses a non-reentrant model
  1141 ;;
  1142                           
  1143                           	psect	text9
  1144  007D30                     __ptext9:
  1145                           	opt stack 0
  1146  007D30                     _NRF24L01_WriteRegister:
  1147                           	opt stack 28
  1148                           
  1149                           ;incstack = 0
  1150                           ;NRF24L01_WriteRegister@Mnemonic stored from wreg
  1151  007D30  6E04               	movwf	NRF24L01_WriteRegister@Mnemonic,c
  1152                           
  1153                           ;nrf24l01.c: 17: LATDbits.LATD1 = 0;
  1154  007D32  928C               	bcf	3980,1,c	;volatile
  1155  007D34                     l1265:
  1156  007D34  5004               	movf	NRF24L01_WriteRegister@Mnemonic,w,c
  1157  007D36  0920               	iorlw	32
  1158  007D38  EC89  F03E         	call	_WriteSPI
  1159  007D3C  0900               	iorlw	0
  1160  007D3E  A4D8               	btfss	status,2,c
  1161  007D40  D7F9               	goto	l1265
  1162  007D42                     l1267:
  1163  007D42  5003               	movf	NRF24L01_WriteRegister@value,w,c
  1164  007D44  EC89  F03E         	call	_WriteSPI
  1165  007D48  0900               	iorlw	0
  1166  007D4A  A4D8               	btfss	status,2,c
  1167  007D4C  D7FA               	goto	l1267
  1168                           
  1169                           ;nrf24l01.c: 20: LATDbits.LATD1 = 1;
  1170  007D4E  828C               	bsf	3980,1,c	;volatile
  1171  007D50  0012               	return		;funcret
  1172  007D52                     __end_of_NRF24L01_WriteRegister:
  1173                           	opt stack 0
  1174                           tblptru	equ	0xFF8
  1175                           tblptrh	equ	0xFF7
  1176                           tblptrl	equ	0xFF6
  1177                           tablat	equ	0xFF5
  1178                           postinc0	equ	0xFEE
  1179                           postdec1	equ	0xFE5
  1180                           fsr1l	equ	0xFE1
  1181                           indf2	equ	0xFDF
  1182                           fsr2h	equ	0xFDA
  1183                           fsr2l	equ	0xFD9
  1184                           status	equ	0xFD8
  1185                           
  1186 ;; *************** function _Delay_ms *****************
  1187 ;; Defined at:
  1188 ;;		line 11 in file "my_delays.c"
  1189 ;; Parameters:    Size  Location     Type
  1190 ;;  count           2    0[COMRAM] unsigned int 
  1191 ;; Auto vars:     Size  Location     Type
  1192 ;;  i               2    3[COMRAM] unsigned int 
  1193 ;; Return value:  Size  Location     Type
  1194 ;;		None               void
  1195 ;; Registers used:
  1196 ;;		wreg, status,2, status,0
  1197 ;; Tracked objects:
  1198 ;;		On entry : 0/0
  1199 ;;		On exit  : 0/0
  1200 ;;		Unchanged: 0/0
  1201 ;; Data sizes:     COMRAM   BANK0   BANK1   BANK2   BANK3   BANK4   BANK5   BANK6   BANK7
  1202 ;;      Params:         2       0       0       0       0       0       0       0       0
  1203 ;;      Locals:         2       0       0       0       0       0       0       0       0
  1204 ;;      Temps:          1       0       0       0       0       0       0       0       0
  1205 ;;      Totals:         5       0       0       0       0       0       0       0       0
  1206 ;;Total ram usage:        5 bytes
  1207 ;; Hardware stack levels used:    1
  1208 ;; This function calls:
  1209 ;;		Nothing
  1210 ;; This function is called by:
  1211 ;;		_NRF24L01_Init
  1212 ;;		_NRF24L01_SendData
  1213 ;;		_NRF24L01_StandbyI
  1214 ;; This function uses a non-reentrant model
  1215 ;;
  1216                           
  1217                           	psect	text10
  1218  007DC0                     __ptext10:
  1219                           	opt stack 0
  1220  007DC0                     _Delay_ms:
  1221                           	opt stack 29
  1222                           
  1223                           ;my_delays.c: 12: unsigned int i;
  1224                           ;my_delays.c: 13: for(i = 0; i < count; i++){
  1225                           
  1226                           ;incstack = 0
  1227  007DC0  0E00               	movlw	0
  1228  007DC2  6E05               	movwf	Delay_ms@i+1,c
  1229  007DC4  0E00               	movlw	0
  1230  007DC6  6E04               	movwf	Delay_ms@i,c
  1231  007DC8  D00A               	goto	l72
  1232  007DCA                     l1271:
  1233                           
  1234                           ;my_delays.c: 14: _delay((unsigned long)((1)*(20000000/4000.0)));
  1235  007DCA  0E07               	movlw	7
  1236  007DCC  6E03               	movwf	??_Delay_ms& (0+255),c
  1237  007DCE  0E7D               	movlw	125
  1238  007DD0                     u397:
  1239  007DD0  2EE8               	decfsz	wreg,f,c
  1240  007DD2  D7FE               	goto	u397
  1241  007DD4  2E03               	decfsz	??_Delay_ms& (0+255),f,c
  1242  007DD6  D7FC               	goto	u397
  1243  007DD8  F000               	nop	
  1244  007DDA  4A04               	infsnz	Delay_ms@i,f,c
  1245  007DDC  2A05               	incf	Delay_ms@i+1,f,c
  1246  007DDE                     l72:
  1247  007DDE  5001               	movf	Delay_ms@count,w,c
  1248  007DE0  5C04               	subwf	Delay_ms@i,w,c
  1249  007DE2  5002               	movf	Delay_ms@count+1,w,c
  1250  007DE4  5805               	subwfb	Delay_ms@i+1,w,c
  1251  007DE6  B0D8               	btfsc	status,0,c
  1252  007DE8  0012               	return	
  1253  007DEA  D7EF               	goto	l1271
  1254  007DEC                     __end_of_Delay_ms:
  1255                           	opt stack 0
  1256                           tblptru	equ	0xFF8
  1257                           tblptrh	equ	0xFF7
  1258                           tblptrl	equ	0xFF6
  1259                           tablat	equ	0xFF5
  1260                           postinc0	equ	0xFEE
  1261                           wreg	equ	0xFE8
  1262                           postdec1	equ	0xFE5
  1263                           fsr1l	equ	0xFE1
  1264                           indf2	equ	0xFDF
  1265                           fsr2h	equ	0xFDA
  1266                           fsr2l	equ	0xFD9
  1267                           status	equ	0xFD8
  1268                           
  1269 ;; *************** function _NRF24L01_DataReady *****************
  1270 ;; Defined at:
  1271 ;;		line 97 in file "nrf24l01.c"
  1272 ;; Parameters:    Size  Location     Type
  1273 ;;		None
  1274 ;; Auto vars:     Size  Location     Type
  1275 ;;		None
  1276 ;; Return value:  Size  Location     Type
  1277 ;;                  1    wreg      unsigned char 
  1278 ;; Registers used:
  1279 ;;		wreg, status,2, status,0, cstack
  1280 ;; Tracked objects:
  1281 ;;		On entry : 0/0
  1282 ;;		On exit  : 0/0
  1283 ;;		Unchanged: 0/0
  1284 ;; Data sizes:     COMRAM   BANK0   BANK1   BANK2   BANK3   BANK4   BANK5   BANK6   BANK7
  1285 ;;      Params:         0       0       0       0       0       0       0       0       0
  1286 ;;      Locals:         0       0       0       0       0       0       0       0       0
  1287 ;;      Temps:          1       0       0       0       0       0       0       0       0
  1288 ;;      Totals:         1       0       0       0       0       0       0       0       0
  1289 ;;Total ram usage:        1 bytes
  1290 ;; Hardware stack levels used:    1
  1291 ;; Hardware stack levels required when called:    2
  1292 ;; This function calls:
  1293 ;;		_NRF24L01_ReadRegister
  1294 ;; This function is called by:
  1295 ;;		_main
  1296 ;; This function uses a non-reentrant model
  1297 ;;
  1298                           
  1299                           	psect	text11
  1300  007CE2                     __ptext11:
  1301                           	opt stack 0
  1302  007CE2                     _NRF24L01_DataReady:
  1303                           	opt stack 28
  1304                           
  1305                           ;nrf24l01.c: 98: if((NRF24L01_ReadRegister(0x07) & 0x40) == 0x40){
  1306                           
  1307                           ;incstack = 0
  1308  007CE2  0E07               	movlw	7
  1309  007CE4  EC7B  F03E         	call	_NRF24L01_ReadRegister
  1310  007CE8  6E05               	movwf	??_NRF24L01_DataReady& (0+255),c
  1311  007CEA  AC05               	btfss	??_NRF24L01_DataReady,6,c
  1312  007CEC  D002               	goto	l1005
  1313                           
  1314                           ;nrf24l01.c: 99: return 0;
  1315  007CEE  0E00               	movlw	0
  1316  007CF0  0012               	return	
  1317  007CF2                     l1005:
  1318                           
  1319                           ;nrf24l01.c: 100: }
  1320                           ;nrf24l01.c: 101: return 1;
  1321  007CF2  0E01               	movlw	1
  1322  007CF4  0012               	return	
  1323  007CF6                     __end_of_NRF24L01_DataReady:
  1324                           	opt stack 0
  1325                           tblptru	equ	0xFF8
  1326                           tblptrh	equ	0xFF7
  1327                           tblptrl	equ	0xFF6
  1328                           tablat	equ	0xFF5
  1329                           postinc0	equ	0xFEE
  1330                           wreg	equ	0xFE8
  1331                           postdec1	equ	0xFE5
  1332                           fsr1l	equ	0xFE1
  1333                           indf2	equ	0xFDF
  1334                           fsr2h	equ	0xFDA
  1335                           fsr2l	equ	0xFD9
  1336                           status	equ	0xFD8
  1337                           
  1338 ;; *************** function _NRF24L01_ReadRegister *****************
  1339 ;; Defined at:
  1340 ;;		line 23 in file "nrf24l01.c"
  1341 ;; Parameters:    Size  Location     Type
  1342 ;;  Mnemonic        1    wreg     unsigned char 
  1343 ;; Auto vars:     Size  Location     Type
  1344 ;;  Mnemonic        1    2[COMRAM] unsigned char 
  1345 ;;  byte0           1    3[COMRAM] unsigned char 
  1346 ;; Return value:  Size  Location     Type
  1347 ;;                  1    wreg      unsigned char 
  1348 ;; Registers used:
  1349 ;;		wreg, status,2, cstack
  1350 ;; Tracked objects:
  1351 ;;		On entry : 0/0
  1352 ;;		On exit  : 0/0
  1353 ;;		Unchanged: 0/0
  1354 ;; Data sizes:     COMRAM   BANK0   BANK1   BANK2   BANK3   BANK4   BANK5   BANK6   BANK7
  1355 ;;      Params:         0       0       0       0       0       0       0       0       0
  1356 ;;      Locals:         2       0       0       0       0       0       0       0       0
  1357 ;;      Temps:          0       0       0       0       0       0       0       0       0
  1358 ;;      Totals:         2       0       0       0       0       0       0       0       0
  1359 ;;Total ram usage:        2 bytes
  1360 ;; Hardware stack levels used:    1
  1361 ;; Hardware stack levels required when called:    1
  1362 ;; This function calls:
  1363 ;;		_ReadSPI
  1364 ;;		_WriteSPI
  1365 ;; This function is called by:
  1366 ;;		_NRF24L01_DataReady
  1367 ;;		_NRF24L01_GetChannel
  1368 ;; This function uses a non-reentrant model
  1369 ;;
  1370                           
  1371                           	psect	text12
  1372  007CF6                     __ptext12:
  1373                           	opt stack 0
  1374  007CF6                     _NRF24L01_ReadRegister:
  1375                           	opt stack 28
  1376                           
  1377                           ;incstack = 0
  1378                           ;NRF24L01_ReadRegister@Mnemonic stored from wreg
  1379  007CF6  6E03               	movwf	NRF24L01_ReadRegister@Mnemonic,c
  1380                           
  1381                           ;nrf24l01.c: 24: unsigned char byte0;
  1382                           ;nrf24l01.c: 25: LATDbits.LATD1 = 0;
  1383  007CF8  928C               	bcf	3980,1,c	;volatile
  1384  007CFA                     l933:
  1385  007CFA  5003               	movf	NRF24L01_ReadRegister@Mnemonic,w,c
  1386  007CFC  EC89  F03E         	call	_WriteSPI
  1387  007D00  0900               	iorlw	0
  1388  007D02  A4D8               	btfss	status,2,c
  1389  007D04  D7FA               	goto	l933
  1390                           
  1391                           ;nrf24l01.c: 27: byte0 = ReadSPI();
  1392  007D06  EC68  F03E         	call	_ReadSPI	;wreg free
  1393  007D0A  6E04               	movwf	NRF24L01_ReadRegister@byte0,c
  1394                           
  1395                           ;nrf24l01.c: 28: LATDbits.LATD1 = 1;
  1396  007D0C  828C               	bsf	3980,1,c	;volatile
  1397                           
  1398                           ;nrf24l01.c: 29: return byte0;
  1399  007D0E  5004               	movf	NRF24L01_ReadRegister@byte0,w,c
  1400  007D10  0012               	return	
  1401  007D12                     __end_of_NRF24L01_ReadRegister:
  1402                           	opt stack 0
  1403                           tblptru	equ	0xFF8
  1404                           tblptrh	equ	0xFF7
  1405                           tblptrl	equ	0xFF6
  1406                           tablat	equ	0xFF5
  1407                           postinc0	equ	0xFEE
  1408                           wreg	equ	0xFE8
  1409                           postdec1	equ	0xFE5
  1410                           fsr1l	equ	0xFE1
  1411                           indf2	equ	0xFDF
  1412                           fsr2h	equ	0xFDA
  1413                           fsr2l	equ	0xFD9
  1414                           status	equ	0xFD8
  1415                           
  1416 ;; *************** function _WriteSPI *****************
  1417 ;; Defined at:
  1418 ;;		line 13 in file "C:\Program Files\Microchip\xc8\v1.35\sources\pic18\plib\SPI\spi_writ.c"
  1419 ;; Parameters:    Size  Location     Type
  1420 ;;  data_out        1    wreg     unsigned char 
  1421 ;; Auto vars:     Size  Location     Type
  1422 ;;  data_out        1    1[COMRAM] unsigned char 
  1423 ;;  TempVar         1    0[COMRAM] unsigned char 
  1424 ;; Return value:  Size  Location     Type
  1425 ;;                  1    wreg      char 
  1426 ;; Registers used:
  1427 ;;		wreg
  1428 ;; Tracked objects:
  1429 ;;		On entry : 0/0
  1430 ;;		On exit  : 0/0
  1431 ;;		Unchanged: 0/0
  1432 ;; Data sizes:     COMRAM   BANK0   BANK1   BANK2   BANK3   BANK4   BANK5   BANK6   BANK7
  1433 ;;      Params:         0       0       0       0       0       0       0       0       0
  1434 ;;      Locals:         2       0       0       0       0       0       0       0       0
  1435 ;;      Temps:          0       0       0       0       0       0       0       0       0
  1436 ;;      Totals:         2       0       0       0       0       0       0       0       0
  1437 ;;Total ram usage:        2 bytes
  1438 ;; Hardware stack levels used:    1
  1439 ;; This function calls:
  1440 ;;		Nothing
  1441 ;; This function is called by:
  1442 ;;		_NRF24L01_WriteRegister
  1443 ;;		_NRF24L01_ReadRegister
  1444 ;;		_NRF24L01_WriteBuffer
  1445 ;;		_NRF24L01_ReadBuffer
  1446 ;;		_NRF24L01_Flush
  1447 ;; This function uses a non-reentrant model
  1448 ;;
  1449                           
  1450                           	psect	text13
  1451  007D12                     __ptext13:
  1452                           	opt stack 0
  1453  007D12                     _WriteSPI:
  1454                           	opt stack 28
  1455                           
  1456                           ;incstack = 0
  1457                           ;WriteSPI@data_out stored from wreg
  1458  007D12  6E02               	movwf	WriteSPI@data_out,c
  1459  007D14  CFC9 F001          	movff	4041,WriteSPI@TempVar	;volatile
  1460  007D18  969E               	bcf	3998,3,c	;volatile
  1461  007D1A  9EC6               	bcf	4038,7,c	;volatile
  1462  007D1C  C002  FFC9         	movff	WriteSPI@data_out,4041	;volatile
  1463  007D20  AEC6               	btfss	4038,7,c	;volatile
  1464  007D22  D002               	goto	l273
  1465  007D24  0EFF               	movlw	255
  1466  007D26  0012               	return	
  1467  007D28                     l273:
  1468  007D28  A69E               	btfss	3998,3,c	;volatile
  1469  007D2A  D7FE               	goto	l273
  1470  007D2C  0E00               	movlw	0
  1471  007D2E  0012               	return	
  1472  007D30                     __end_of_WriteSPI:
  1473                           	opt stack 0
  1474                           tblptru	equ	0xFF8
  1475                           tblptrh	equ	0xFF7
  1476                           tblptrl	equ	0xFF6
  1477                           tablat	equ	0xFF5
  1478                           postinc0	equ	0xFEE
  1479                           wreg	equ	0xFE8
  1480                           postdec1	equ	0xFE5
  1481                           fsr1l	equ	0xFE1
  1482                           indf2	equ	0xFDF
  1483                           fsr2h	equ	0xFDA
  1484                           fsr2l	equ	0xFD9
  1485                           status	equ	0xFD8
  1486                           
  1487 ;; *************** function _ReadSPI *****************
  1488 ;; Defined at:
  1489 ;;		line 12 in file "C:\Program Files\Microchip\xc8\v1.35\sources\pic18\plib\SPI\spi_read.c"
  1490 ;; Parameters:    Size  Location     Type
  1491 ;;		None
  1492 ;; Auto vars:     Size  Location     Type
  1493 ;;  TempVar         1    0[COMRAM] unsigned char 
  1494 ;; Return value:  Size  Location     Type
  1495 ;;                  1    wreg      unsigned char 
  1496 ;; Registers used:
  1497 ;;		wreg, status,2
  1498 ;; Tracked objects:
  1499 ;;		On entry : 0/0
  1500 ;;		On exit  : 0/0
  1501 ;;		Unchanged: 0/0
  1502 ;; Data sizes:     COMRAM   BANK0   BANK1   BANK2   BANK3   BANK4   BANK5   BANK6   BANK7
  1503 ;;      Params:         0       0       0       0       0       0       0       0       0
  1504 ;;      Locals:         1       0       0       0       0       0       0       0       0
  1505 ;;      Temps:          0       0       0       0       0       0       0       0       0
  1506 ;;      Totals:         1       0       0       0       0       0       0       0       0
  1507 ;;Total ram usage:        1 bytes
  1508 ;; Hardware stack levels used:    1
  1509 ;; This function calls:
  1510 ;;		Nothing
  1511 ;; This function is called by:
  1512 ;;		_NRF24L01_ReadRegister
  1513 ;;		_NRF24L01_ReadBuffer
  1514 ;; This function uses a non-reentrant model
  1515 ;;
  1516                           
  1517                           	psect	text14
  1518  007CD0                     __ptext14:
  1519                           	opt stack 0
  1520  007CD0                     _ReadSPI:
  1521                           	opt stack 28
  1522                           
  1523                           ;incstack = 0
  1524  007CD0  CFC9 F001          	movff	4041,ReadSPI@TempVar	;volatile
  1525  007CD4  969E               	bcf	3998,3,c	;volatile
  1526  007CD6  0E00               	movlw	0
  1527  007CD8  6EC9               	movwf	4041,c	;volatile
  1528  007CDA                     l256:
  1529  007CDA  A69E               	btfss	3998,3,c	;volatile
  1530  007CDC  D7FE               	goto	l256
  1531  007CDE  50C9               	movf	4041,w,c	;volatile
  1532  007CE0  0012               	return	
  1533  007CE2                     __end_of_ReadSPI:
  1534                           	opt stack 0
  1535  0000                     tblptru	equ	0xFF8
  1536                           tblptrh	equ	0xFF7
  1537                           tblptrl	equ	0xFF6
  1538                           tablat	equ	0xFF5
  1539                           postinc0	equ	0xFEE
  1540                           wreg	equ	0xFE8
  1541                           postdec1	equ	0xFE5
  1542                           fsr1l	equ	0xFE1
  1543                           indf2	equ	0xFDF
  1544                           fsr2h	equ	0xFDA
  1545                           fsr2l	equ	0xFD9
  1546                           status	equ	0xFD8
  1547                           tblptru	equ	0xFF8
  1548                           tblptrh	equ	0xFF7
  1549                           tblptrl	equ	0xFF6
  1550                           tablat	equ	0xFF5
  1551                           postinc0	equ	0xFEE
  1552                           wreg	equ	0xFE8
  1553                           postdec1	equ	0xFE5
  1554                           fsr1l	equ	0xFE1
  1555                           indf2	equ	0xFDF
  1556                           fsr2h	equ	0xFDA
  1557                           fsr2l	equ	0xFD9
  1558                           status	equ	0xFD8
  1559                           
  1560                           	psect	rparam
  1561  0000                     tblptru	equ	0xFF8
  1562                           tblptrh	equ	0xFF7
  1563                           tblptrl	equ	0xFF6
  1564                           tablat	equ	0xFF5
  1565                           postinc0	equ	0xFEE
  1566                           wreg	equ	0xFE8
  1567                           postdec1	equ	0xFE5
  1568                           fsr1l	equ	0xFE1
  1569                           indf2	equ	0xFDF
  1570                           fsr2h	equ	0xFDA
  1571                           fsr2l	equ	0xFD9
  1572                           status	equ	0xFD8


Data Sizes:
    Strings     0
    Constant    0
    Data        5
    BSS         0
    Persistent  0
    Stack       0

Auto Spaces:
    Space          Size  Autos    Used
    COMRAM           95     41      46
    BANK0           160      0       0
    BANK1           256      0       0
    BANK2           256      0       0
    BANK3           256      0       0
    BANK4           256      0       0
    BANK5           256      0       0
    BANK6           256      0       0
    BANK7           256      0       0

Pointer List with Targets:

    NRF24L01_ReadData@buffer	PTR unsigned char  size(2) Largest target is 32
		 -> main@bufferRX(COMRAM[32]), 

    NRF24L01_ReadBuffer@buffer	PTR unsigned char  size(2) Largest target is 32
		 -> main@bufferRX(COMRAM[32]), 

    NRF24L01_WriteBuffer@buffer	PTR unsigned char  size(2) Largest target is 5
		 -> ADDRESS_DATA_PIPE0(COMRAM[5]), 


Critical Paths under _main in COMRAM

    _main->_NRF24L01_Init
    _main->_NRF24L01_ReadData
    _NRF24L01_ReadData->_NRF24L01_ReadBuffer
    _NRF24L01_ReadBuffer->_WriteSPI
    _NRF24L01_Init->_NRF24L01_WriteBuffer
    _NRF24L01_WriteBuffer->_WriteSPI
    _NRF24L01_SetMode->_NRF24L01_WriteRegister
    _NRF24L01_Flush->_WriteSPI
    _NRF24L01_SetChannel->_NRF24L01_WriteRegister
    _NRF24L01_WriteRegister->_WriteSPI
    _NRF24L01_DataReady->_NRF24L01_ReadRegister
    _NRF24L01_ReadRegister->_WriteSPI

Critical Paths under _main in BANK0

    None.

Critical Paths under _main in BANK1

    None.

Critical Paths under _main in BANK2

    None.

Critical Paths under _main in BANK3

    None.

Critical Paths under _main in BANK4

    None.

Critical Paths under _main in BANK5

    None.

Critical Paths under _main in BANK6

    None.

Critical Paths under _main in BANK7

    None.

Call Graph Tables:

 ---------------------------------------------------------------------------------
 (Depth) Function   	        Calls       Base Space   Used Autos Params    Refs
 ---------------------------------------------------------------------------------
 (0) _main                                                32    32      0    5317
                                              9 COMRAM    32    32      0
                 _NRF24L01_DataReady
                      _NRF24L01_Init
                  _NRF24L01_ReadData
                            _OpenSPI
 ---------------------------------------------------------------------------------
 (1) _OpenSPI                                              3     1      2     216
                                              0 COMRAM     3     1      2
 ---------------------------------------------------------------------------------
 (1) _NRF24L01_ReadData                                    2     0      2    1248
                                              7 COMRAM     2     0      2
                     _NRF24L01_Flush
                _NRF24L01_ReadBuffer
             _NRF24L01_WriteRegister
 ---------------------------------------------------------------------------------
 (2) _NRF24L01_ReadBuffer                                  5     2      3     256
                                              2 COMRAM     5     2      3
                            _ReadSPI
                           _WriteSPI
 ---------------------------------------------------------------------------------
 (1) _NRF24L01_Init                                        2     1      1    3760
                                              7 COMRAM     2     1      1
                           _Delay_ms
                _NRF24L01_SetChannel
                   _NRF24L01_SetMode
               _NRF24L01_WriteBuffer
             _NRF24L01_WriteRegister
 ---------------------------------------------------------------------------------
 (2) _NRF24L01_WriteBuffer                                 5     2      3     490
                                              2 COMRAM     5     2      3
                           _WriteSPI
 ---------------------------------------------------------------------------------
 (2) _NRF24L01_SetMode                                     1     1      0     928
                                              4 COMRAM     1     1      0
                     _NRF24L01_Flush
             _NRF24L01_WriteRegister
 ---------------------------------------------------------------------------------
 (2) _NRF24L01_Flush                                       0     0      0      15
                           _WriteSPI
 ---------------------------------------------------------------------------------
 (2) _NRF24L01_SetChannel                                  1     1      0     913
                                              4 COMRAM     1     1      0
             _NRF24L01_WriteRegister
 ---------------------------------------------------------------------------------
 (2) _NRF24L01_WriteRegister                               2     1      1     891
                                              2 COMRAM     2     1      1
                           _WriteSPI
 ---------------------------------------------------------------------------------
 (2) _Delay_ms                                             5     3      2     430
                                              0 COMRAM     5     3      2
 ---------------------------------------------------------------------------------
 (1) _NRF24L01_DataReady                                   1     1      0      45
                                              4 COMRAM     1     1      0
              _NRF24L01_ReadRegister
 ---------------------------------------------------------------------------------
 (2) _NRF24L01_ReadRegister                                2     2      0      45
                                              2 COMRAM     2     2      0
                            _ReadSPI
                           _WriteSPI
 ---------------------------------------------------------------------------------
 (3) _WriteSPI                                             2     2      0      15
                                              0 COMRAM     2     2      0
 ---------------------------------------------------------------------------------
 (3) _ReadSPI                                              1     1      0       0
                                              0 COMRAM     1     1      0
 ---------------------------------------------------------------------------------
 Estimated maximum stack depth 3
 ---------------------------------------------------------------------------------

 Call Graph Graphs:

 _main (ROOT)
   _NRF24L01_DataReady
     _NRF24L01_ReadRegister
       _ReadSPI
       _WriteSPI
   _NRF24L01_Init
     _Delay_ms
     _NRF24L01_SetChannel
       _NRF24L01_WriteRegister
         _WriteSPI
     _NRF24L01_SetMode
       _NRF24L01_Flush
         _WriteSPI
       _NRF24L01_WriteRegister
         _WriteSPI
     _NRF24L01_WriteBuffer
       _WriteSPI
     _NRF24L01_WriteRegister
       _WriteSPI
   _NRF24L01_ReadData
     _NRF24L01_Flush
       _WriteSPI
     _NRF24L01_ReadBuffer
       _ReadSPI
       _WriteSPI
     _NRF24L01_WriteRegister
       _WriteSPI
   _OpenSPI

 Address spaces:
Name               Size   Autos  Total    Cost      Usage
BIGRAM             7FF      0       0      21        0.0%
EEDATA             100      0       0       0        0.0%
BITBANK7           100      0       0      18        0.0%
BANK7              100      0       0      19        0.0%
BITBANK6           100      0       0      16        0.0%
BANK6              100      0       0      17        0.0%
BITBANK5           100      0       0      14        0.0%
BANK5              100      0       0      15        0.0%
BITBANK4           100      0       0      12        0.0%
BANK4              100      0       0      13        0.0%
BITBANK3           100      0       0      10        0.0%
BANK3              100      0       0      11        0.0%
BITBANK2           100      0       0       8        0.0%
BANK2              100      0       0       9        0.0%
BITBANK1           100      0       0       6        0.0%
BANK1              100      0       0       7        0.0%
BITBANK0            A0      0       0       4        0.0%
BANK0               A0      0       0       5        0.0%
BITCOMRAM           5F      0       0       0        0.0%
COMRAM              5F     29      2E       1       48.4%
BITSFR               0      0       0      40        0.0%
SFR                  0      0       0      40        0.0%
STACK                0      0       0       2        0.0%
NULL                 0      0       0       0        0.0%
ABS                  0      0      2E      20        0.0%
DATA                 0      0      2E       3        0.0%
CODE                 0      0       0       0        0.0%


Microchip Technology PIC18 Macro Assembler V1.35 build -356382666 
Symbol Table                                                                                   Thu Apr 27 03:08:27 2017

                    _SSPSTATbits 000FC7                               l72 7DDE  
                    __CFG_BOR$ON 000000                      __CFG_BORV$3 000000  
                   __CFG_CP0$OFF 000000                     __CFG_CP1$OFF 000000  
                            l241 7F10                              l242 7F12  
                            l219 7EF6                              l245 7F2C  
                            l246 7F46                              l247 7F2E  
                            l239 7F0C                              l256 7CDA  
                            l248 7F32                              l273 7D28  
                            l921 7D54                              l923 7D64  
                            l933 7CFA                     __CFG_CPB$OFF 000000  
                            u397 7DD0                              wreg 000FE8  
           _NRF24L01_WriteBuffer 7DEC                    _NRF24L01_Init 7F4E  
                   __CFG_LVP$OFF 000000                     __CFG_WDT$OFF 000000  
                           l1005 7CF2                             l1311 7E3A  
                           l1321 7E56                             l1315 7E48  
                           l1271 7DCA                             l1351 7F36  
                           l1265 7D34                             l1281 7E02  
                           l1267 7D42                             l1347 7F16  
                           l1285 7E1C                             l1277 7DF0  
                           l1293 7E7C                             l1289 7E6A  
                           l1377 7EDA                             l1299 7E90  
                           _LATB 000F8A  __size_of_NRF24L01_WriteRegister 0022  
                           _main 7EA8                             fsr2h 000FDA  
                           fsr1l 000FE1                             indf2 000FDF  
                           fsr2l 000FD9                             start 1000  
                  __CFG_IESO$OFF 000000                    __CFG_MCLRE$ON 000000  
                   ___param_bank 000010    NRF24L01_SetChannel@rf_channel 0005  
                __end_of_ReadSPI 7CE2                   _NRF24L01_Flush 7D52  
                __end_of_OpenSPI 7F4E             NRF24L01_ReadBuffer@i 0007  
      NRF24L01_ReadBuffer@buffer 0003                    __CFG_PLLDIV$5 000000  
                   main@bufferRX 000A                            ?_main 0001  
                  __CFG_USBDIV$2 000000         NRF24L01_WriteBuffer@data 0006  
                          _TRISB 000F93                            _TRISD 000F95  
          ?_NRF24L01_WriteBuffer 0003                    __CFG_PWRT$OFF 000000  
                  __CFG_WRT0$OFF 000000                    __CFG_WRT1$OFF 000000  
                 __CFG_EBTR0$OFF 000000                   __CFG_FCMEN$OFF 000000  
                 __CFG_EBTR1$OFF 000000                   ?_NRF24L01_Init 0008  
                  __CFG_WRTB$OFF 000000                    __CFG_WRTC$OFF 000000  
      __size_of_NRF24L01_SetMode 003E                   __CFG_EBTRB$OFF 000000  
                          tablat 000FF5                            status 000FD8  
               __end_of_Delay_ms 7DEC           __end_of_NRF24L01_Flush 7D74  
                __initialization 7D96                     __end_of_main 7EF8  
             _NRF24L01_DataReady 7CE2           _NRF24L01_WriteRegister 7D30  
   __size_of_NRF24L01_ReadBuffer 0042                           ??_main 000A  
                  __activetblptr 000002              ?_NRF24L01_DataReady 0001  
                         _ADCON0 000FC2                           _ADCON1 000FC1  
   __size_of_NRF24L01_SetChannel 000E                 __end_of_WriteSPI 7D30  
 __size_of_NRF24L01_ReadRegister 001C    __end_of_NRF24L01_ReadRegister 7D12  
                         _SSPBUF 000FC9             ??_NRF24L01_DataReady 0005  
                      ??_ReadSPI 0001                   __CFG_VREGEN$ON 000000  
                      ??_OpenSPI 0003                   __CFG_XINST$OFF 000000  
                ?_NRF24L01_Flush 0001                   __CFG_STVREN$ON 000000  
                  Delay_ms@count 0001                  WriteSPI@TempVar 0001  
         ??_NRF24L01_WriteBuffer 0006                  ??_NRF24L01_Init 0009  
                   __pdataCOMRAM 002A                           tblptrh 000FF7  
                         tblptrl 000FF6                           tblptru 000FF8  
           NRF24L01_SetMode@mode 0005         NRF24L01_ReadBuffer@bytes 0005  
                     __accesstop 0060          __end_of__initialization 7DB6  
                __CFG_PBADEN$OFF 000000                    ___rparam_used 000001  
          NRF24L01_WriteBuffer@i 0007                   __pcstackCOMRAM 0001  
                      ?_Delay_ms 0001                 _NRF24L01_SetMode 7E28  
  NRF24L01_ReadRegister@Mnemonic 0003                        ?_WriteSPI 0001  
                     ??_Delay_ms 0003                          _SSPCON1 000FC6  
                        _SSPSTAT 000FC7              _NRF24L01_ReadBuffer 7E66  
                        _ReadSPI 7CD0                          _OpenSPI 7EF8  
                        __Hparam 0000          ?_NRF24L01_WriteRegister 0003  
                        __Lparam 0000              _NRF24L01_SetChannel 7CC2  
           ?_NRF24L01_ReadBuffer 0003                          __pcinit 7D96  
        NRF24L01_Init@rf_channel 0008                          __ramtop 0800  
                     ??_WriteSPI 0001                          __ptext0 7EA8  
                        __ptext1 7EF8                          __ptext2 7D74  
                        __ptext3 7E66                          __ptext4 7F4E  
                        __ptext5 7DEC                          __ptext6 7E28  
                        __ptext7 7D52                          __ptext8 7CC2  
                        __ptext9 7D30             ?_NRF24L01_SetChannel 0001  
           end_of_initialization 7DB6                        Delay_ms@i 0004  
               ??_NRF24L01_Flush 0003                    __Lmediumconst 0000  
 __end_of_NRF24L01_WriteRegister 7D52                          postdec1 000FE5  
               WriteSPI@data_out 0002                          postinc0 000FEE  
          ??_NRF24L01_ReadBuffer 0006      NRF24L01_WriteRegister@value 0003  
                      _TRISAbits 000F92                        _TRISBbits 000F93  
                      _TRISCbits 000F94                        _TRISDbits 000F95  
        NRF24L01_ReadData@buffer 0008            ??_NRF24L01_SetChannel 0005  
              NRF24L01_Init@mode 0009       NRF24L01_ReadRegister@byte0 0004  
    __size_of_NRF24L01_DataReady 0014            _NRF24L01_ReadRegister 7CF6  
       __end_of_NRF24L01_SetMode 7E66                    __pidataCOMRAM 7CBD  
               OpenSPI@smp_phase 0002       NRF24L01_WriteBuffer@buffer 0003  
            start_initialization 7D96    __size_of_NRF24L01_WriteBuffer 003C  
                 ReadSPI@TempVar 0001            __end_of_NRF24L01_Init 8000  
              __size_of_Delay_ms 002C                 OpenSPI@sync_mode 0003  
              _NRF24L01_ReadData 7D74               ?_NRF24L01_ReadData 0008  
               __CFG_LPT1OSC$OFF 000000              ??_NRF24L01_ReadData 000A  
        NRF24L01_ReadBuffer@data 0006                __size_of_WriteSPI 001E  
      __end_of_NRF24L01_ReadData 7D96           ?_NRF24L01_ReadRegister 0001  
                       ?_ReadSPI 0001                         ?_OpenSPI 0001  
 NRF24L01_WriteRegister@Mnemonic 0004                         _LATDbits 000F8C  
                       _PIR1bits 000F9E                 __CFG_WDTPS$32768 000000  
                OpenSPI@bus_mode 0001                       _ADCON1bits 000FC1  
                       _Delay_ms 7DC0                        copy_data0 7DAA  
      NRF24L01_WriteBuffer@bytes 0005       __size_of_NRF24L01_ReadData 0022  
    __end_of_NRF24L01_ReadBuffer 7EA8                 __size_of_ReadSPI 0012  
                       __Hrparam 0000               _ADDRESS_DATA_PIPE0 002A  
                       __Lrparam 0000                 __size_of_OpenSPI 0056  
              ?_NRF24L01_SetMode 0001               ??_NRF24L01_SetMode 0005  
                       _WriteSPI 7D12      __end_of_NRF24L01_SetChannel 7CD0  
                       __ptext10 7DC0                         __ptext11 7CE2  
                       __ptext12 7CF6                         __ptext13 7D12  
                       __ptext14 7CD0       __end_of_NRF24L01_DataReady 7CF6  
                  __size_of_main 0050     __end_of_NRF24L01_WriteBuffer 7E28  
        __size_of_NRF24L01_Flush 0022            __CFG_CPUDIV$OSC1_PLL2 000000  
       ??_NRF24L01_WriteRegister 0004          ??_NRF24L01_ReadRegister 0003  
         __size_of_NRF24L01_Init 00B2                      _SSPCON1bits 000FC6  
             __CFG_FOSC$HSPLL_HS 000000  
